:100000000C949E060C94F1080C94E5060C94E506FD
:100010000C94E5060C94E5060C94E5060C94E506B4
:100020000C94E5060C94E5060C9408260C94DC264A
:100030000C94DC1C0C94E5060C94E5060C94E50687
:100040000C94E5060C94E5060C94E5060C94E50684
:100050000C94E5060C94421D0C94E5060C94E50600
:100060000C94E5060C94E5060C94E5060C94E50664
:100070000C94E5060C94E5060C94E5060C94E50654
:100080000C94E5060C94E5060C94E5060C94E50644
:100090000C94E5060C94E5060C94E5060C94E50634
:1000A0000C94E5060C94E5060C94E50601E301E0EA
:1000B000014F024F02E002E30001E301E0015002C0
:1000C0005002E002E30001E30115021574FF02E3B0
:1000D00074FF010602060110021001070207012841
:1000E000022874FF01130213010C020C011102110A
:1000F000010A020A012C022C01E00119021902E096
:100100000001E30115021502E301060206011002D7
:1001100010010702070128022874FF74FF010C0276
:100120000C01130213010602060112021201110250
:100130001101090209010C020C010A020A012C0238
:100140002C0138023801040204010F020F010F02D2
:100150000F012802280001E30115021574FF02E3D4
:1001600074FF0106020601100210010702070128B0
:1001700002280001E0010402040106020602E00078
:1001800001E00119021902E00001E0010602060285
:10019000E000757365726E616D65012B706173733C
:1001A000012B012800750A012B022B010C020C0106
:1001B000110211012B022B01280228012B022B0115
:1001C0002B022B012B022B010C020C01110211013D
:1001D0002B022B0128022800750A012B022B011289
:1001E000021201170217012B022B01280228012BF2
:1001F000022B012B022B012B022B011D021D0115CD
:100200000215012B022B0128022800750A012B027E
:100210002B0112021201130213012B022B012802DF
:1002200028012B022B012B022B012B022B011D027B
:100230001D01150215012B022B01280228006970EF
:10024000636F6E666967202F616C6C0000750A0130
:1002500027022701060206012B022B012B022B018C
:10026000040204012B022B00011B021B00750A0172
:10027000E001170217011902190128022802E00003
:100280007777772E737570706F72742E7865726FD2
:10029000782E636F6D012800656D61696C00750AC9
:1002A000010402040107020701100210010C020CF4
:1002B00001110211744B012B022B011E021E011EA3
:1002C000021E011E021E011E021E0128022800013C
:1002D000E3012B022B02E30014001A0008001500B2
:1002E0001700000004001600070009000A000000C3
:1002F0001D001B0006001900050000004D004A000B
:10030000E2002961000000004C002A00000000000B
:1003100000000000130012000C0018001C00000078
:1003200033000F000E000D000B00000038003700F6
:1003300036001000110000004E004B00E300E40006
:100340000000000028002C00000000000000000059
:1003500014001A00090013000A0000000400150030
:1003600016001700070000001D001B000600190002
:10037000050000004D004A00E20029610000000075
:100380004C002A00000000000000000033001C00A8
:1003900018000F000D00000012000C0008001100F2
:1003A0000B00000038003700360010000E0000007F
:1003B0004E004B00E300E4000000000028002C0089
:1003C0000000000000000000340036003700130079
:1003D0001C00000004001200080018000C000000BF
:1003E000330014000D000E001B0000004D004A00F9
:1003F000E2002961000000004C002A00000000001B
:10040000000000000F00150006000A0009000000AF
:100410001600110017000B00070000001D00190056
:100420001A001000050000004E004B00E300E4003D
:100430000000000028002C00000000000000000068
:1004400001000330023001000F30000006300100CF
:100450000100010001000000005C0130010001000A
:1004600001000000003046004E004B00000000007C
:10047000E1002A0000000000000000000A30010036
:10048000010001000100000001000B3052000100DA
:1004900001000000005C4F0051005000010000000E
:1004A000DE5C4C004A004D000000000028002C00DB
:1004B00000000000000000001E0003301E001E00AF
:1004C0001E0000001E001E001E001E001E00000078
:1004D000005C1E001E001E001E00000000304600D2
:1004E0004E004B0000000000E1002A000000000068
:1004F0000000000056002300220021000000000040
:10050000570020001F001E00000000000000370000
:100510002700270000000000DE5C4C004A004D0070
:100520000000000028002C00000000000000000077
:1005300020002000200020002000000001005200C8
:100540000100010001000000500051004F000100B7
:1005500001000000003046004E004B00000000008B
:10056000DD5C2A0000000000000000000100010026
:100570000100010001000000010052000100010023
:10058000010000004F005100500001000100000078
:10059000DE5C4C004D004A000000000028002C00EA
:1005A000000000000000000000000000000000004B
:1005B000000000000000000000000000000000003B
:1005C000000000000000000000000000000000002B
:1005D000000000000000000000000000000000001B
:100A50000000000000000000DB5CDC5CDA5CC15CD4
:100A6000C45C0000DB5C01001D5C1E5C135C0000CC
:100A700001000100DA5C010001000000010001003A
:100A80000100010000000000010001000000000062
:100A900000000000C75CC85CC55CC65CC35C0000AD
:100AA0000100DC5CDA5CDB5C0A5C0000005C0100DD
:100AB000010001000100000001000100010001002F
:100AC0000000000001000100000000000000000024
:100AD00000000000000000002A2B28000000000099
:100AE00000000000000000000000002900000000DD
:100AF0002C1E3420212224342627252E362D37384B
:100B0000271E1F202122232425263333362E373853
:100B10001F0405060708090A0B0C0D0E0F10111211
:100B2000131415161718191A1B1C1D2F3130232DDD
:100B3000350405060708090A0B0C0D0E0F101112DB
:100B4000131415161718191A1B1C1D2F3130354C8C
:100B50000000000000000000000000000000000095
:100B60000000000000000000000000000000000085
:100B7000000101010101010001010101000000006B
:100B80000000000000000000000001000100010161
:100B90000101010101010101010101010101010145
:100BA0000101010101010101010101000000010138
:100BB0000000000000000000000000000000000035
:100BC0000000000000000000000000010101010021
:100BD0000403300000001603520065006E0074002C
:100BE00061006C00200043006100720000001E03E1
:100BF0002F0075002F0063007200790073007400ED
:100C000061006C00680061006E0064000000040375
:100C1000090409025400030100A0FA0904000001BC
:100C20000301010009211101000122400007058193
:100C30000308000A0904010001030102000921114F
:100C4000010001224D000705820308000A09040281
:100C500000010300000009211101000122360007F4
:100C600005830308000A1201100100000008EDFED0
:100C7000603001000102030105010980A101850224
:100C80001601002603001A81002A830075109501C1
:100C90008100C0050C0901A1018503160100269CF5
:100CA000021A01002A9C02751095018100C00501FD
:100CB0000902A1010901A100050919012905150071
:100CC00025019505750181029501750381010501D5
:100CD000093009311581257F95027508810609388B
:100CE0001581257F950175088106050C0A380215C6
:100CF00081257F950175088106C0C005010906A1FF
:100D000001050719E029E7150025019508750181FE
:100D100002950175088101050819012905950575D8
:100D20000191029501750391010507190029FF152D
:100D30000026FF00950675088100C00011241FBE23
:100D4000CFEFDAE0DEBFCDBF04B603FE27C080914F
:100D50004F0290915002A0915102B09152028730FF
:100D6000904BA740B04BD1F410924F02109250021A
:100D7000109251021092520214BE84B7877F84BF32
:100D80000FB6F894A8958091600088618093600008
:100D9000109260000FBEE0E0F8E3099511E0A0E0DA
:100DA000B1E0E6EAF2E502C005900D92AE38B10777
:100DB000D9F722E0AEE8B1E001C01D92AF34B2072E
:100DC000E1F70E9435230C94F2280C9400000C9457
:100DD0007C0A809122028B6080932202ABE6B1E014
:100DE00061E070E08D91E82FE295EF70F0E041A1B5
:100DF0008F709B0101C0220F8A95EAF7922F909580
:100E0000942391A382A1822B82A381E0A037B8070B
:100E100049F7A5E6B1E061E070E08D91E82FE29539
:100E2000EF70F0E041A18F709B0101C0220F8A9505
:100E3000EAF7922F9095942391A382A1822B82A30B
:100E400081E0AB36B80749F7559A209AEEE8F1E011
:100E5000A9E9B1E088E991E011921D928E179F07F0
:100E6000D9F70C94180D3F924F925F926F927F9238
:100E70008F929F92AF92BF92CF92DF92EF92FF92AA
:100E80000F931F93CF93DF9300D000D0CDB7DEB781
:100E9000809100018111B0C085E090E09A83898340
:100EA00009811A8107561E4F8BE6E82E81E0F82E45
:100EB0006801AA24A394B12C8824839424E0922E60
:100EC000D6016D906D01FD011292FC83EB83D70179
:100ED0008D917D01E82FE295EF70F0E091A18F7088
:100EE000B50101C0660F8A95EAF7892F862B81A389
:100EF00082A1762E7094872182A3B0EABA95F1F789
:100F000045E651E090E080E0DA015D90AD01252DED
:100F100022952F7030E0D90190963C90AB81BC8136
:100F20004C90352D3F70D50102C0AA0FBB1F3A95DA
:100F3000E2F79D01232109F062C02A2D082E01C08D
:100F4000220F0A94EAF72429AB81BC812C930196E5
:100F500086309105C9F681A1782271A282A1682B01
:100F600062A38C91681659F08092A3010E940C1D17
:100F70009093A5018093A4018BB189258BB9B0E72B
:100F8000EB16B1E0FB0609F09BCF8091A30188230B
:100F9000E1F08091A4019091A5010E94181D06978F
:100FA000A0F0E981FA81E257FE4FFA83E98380E0FD
:100FB000D8019D918D01E981FA819193FA83E983AA
:100FC0008F5F8530A9F71092A30181E00F900F90F9
:100FD0000F900F90DF91CF911F910F91FF90EF90A5
:100FE000DF90CF90BF90AF909F908F907F906F9049
:100FF0005F904F903F9008951A82198251CF20E060
:10100000A2CFCF93DF9380910001D0E0C0E088238E
:1010100011F0C5E0D0E00E945609009789F4C2574C
:10102000DE4F30E020E0F901E855FE4F4081499362
:101030002F5F3F4F25303105B1F7DF91CF910895F4
:1010400081E090E0FACFCF930E943307C82F0E942F
:101050000108892BE1F05D98809198018F5F809362
:101060009801863078F080910001F0E0E0E088237C
:1010700011F0E5E0F0E0E257FE4F1082118212829B
:10108000138214820E941A0D8C2FCF9108955D9ABD
:1010900010929801F7CF0E94330780910001E5E09C
:1010A000F0E0882311F0F0E0E0E0E257FE4F90E03E
:1010B00080E02191DC01A855BE4F2C93019685302C
:1010C0009105B9F70895E82FF0E0E257FE4F8081CF
:1010D00008950895E8EDF0E08081806180838AE1E1
:1010E0008A95F1F700C08091D900817008958EE053
:1010F00090E00E94BC2891E0811101C090E09093A3
:1011000000010E946A08882321F00E94E408789474
:1011100008950E94031D0E94E808F9CF0E94E90685
:101120000E944B08FDCF0E9477080E946A08811137
:1011300002C00E948E080895509A08955098589AB7
:101140000895589A08950E949E08489BFECF80E813
:101150008A95F1F708950E949E0898E080E029B1F1
:10116000880F2170822B20E82A95F1F725E02A9537
:10117000F1F70000915099F708950F931F93CF93C3
:10118000082F0E949C08C8E010E0C15020F4CF91C5
:101190001F910F910895C8010C2E02C09595879557
:1011A0000A94E2F780FF06C00E94A10880E88A95B1
:1011B000F1F7EBCF5898FACF0E949C08589880E836
:1011C0008A95F1F70C94A1080E949C080C94A10840
:1011D0000E949E08E89AE9E6F0E080818C7F808397
:1011E00008951F920F920FB60F921124EF92FF9263
:1011F0001F932F933F934F935F936F937F938F939F
:101200009F93AF93BF93CF93DF93EF93FF930E948E
:10121000DC08D0E0C0E010E0CE0188559E4F7C0194
:10122000FC0180810E94BD080E94DC08F7018081DA
:10123000180F2196C530D10579F7812F0E94BD087E
:101240000E94DC08F0E8FA95F1F780E48A95F1F75E
:101250000E94AB088093A7010E94DC08D091A701EF
:101260000E94AB08C82F0E94DC080E949E08809153
:10127000A601DC17C9F081608093A601FF91EF9170
:10128000DF91CF91BF91AF919F918F917F916F919E
:101290005F914F913F912F911F91FF90EF900F9091
:1012A0000FBE0F901F9018958E7FE6CFEF92FF92A2
:1012B0001F93CF93DF93F8940E949C08589825E0E1
:1012C0002A95F1F700000E949E080E94A10830E8CC
:1012D0003A95F1F789B1182F117080FF09C0789401
:1012E00081E090E0DF91CF911F91FF90EF90089502
:1012F0000E94A308D0E0C0E00E94AB08FE01E855C0
:10130000FE4F7F0180830E94A308F7018081180FA0
:101310002196C530D10581F70E94AB08C82F0E94E5
:10132000A3081C13DCCF8091A7010E94BD080E9476
:10133000A3088091A7010E94BD080E94A3080E94F3
:101340009C080E94A108789490E080E0CBCF0C9498
:101350007B0AFC018081813021F489E891E00C94C2
:101360008F19823019F480E891E0F9CF83E791E09A
:10137000F6CFFC018081813021F486E591E00C9468
:101380008F19823019F481E091E0F9CF86EC90E07A
:10139000F6CFFC018081813021F489EB90E00C9440
:1013A0008F19823019F48CEA90E0F9CF0895FC018E
:1013B0008081813031F488E30E944F1288E30C94DD
:1013C0002A1381E30E944F1281E3F9CFCF93DF9379
:1013D000EC010E94451CBE0190E080E0DF91CF91BE
:1013E0000C94151ADC016031C8F4E62FF0E0EC50E3
:1013F000F74D0C94A22812968C911297811163C01C
:1014000012968C911297811161C012968C9112974D
:10141000882339F088E992E00E94AF0C90E080E0E8
:10142000089512968C911297882319F080E892E023
:10143000F3CF12968C91129781114BC015968C9117
:101440001597982F907F12962C91222341F0992383
:1014500011F080FFE3CF83E00E94771ADFCF99235A
:1014600011F080FF39C083E00E94981AD7CF1296FE
:101470008C911297811133C012968C911297882308
:1014800019F08CE492E0C8CF12968C9112978823C1
:1014900019F08EE392E0C0CF12968C9112978111D1
:1014A00021C012968C91129781111FC012968C91B7
:1014B000129781111DC012968C91882309F4AECF2A
:1014C00082E991E0A9CF8FEC92E008958EE992E055
:1014D00008958DE692E0089588E692E008958DE4FF
:1014E00092E008958BE092E0089588ED91E00895F0
:1014F00085EA91E0089508950895CF93FB018C3D0E
:101500002CE5920751F158F48A3D2CE59207B1F091
:101510008B3D9C45E1F0C1E08C2FCF9108958E3D2D
:101520002CE5920761F1F8F0803E9C45A1F7C2815D
:1015300080E1CC2379F10E94771A07C0C28182E052
:1015400090E0CC2349F30E94E609C0E0E5CFC281D8
:1015500081E090E0CC2301F3F6CFC281CC23E1F20D
:1015600084E090E0F0CFC28183E0CC2359F00E9468
:10157000771A40E164E083E00E94060DE6CFC28165
:1015800084E0F3CF0E94981A40E164E083E00E9477
:10159000060DC2CF0E94981ABFCF81E008950C9427
:1015A0007D0A0E941F162FEF84E39CE021508040AB
:1015B0009040E1F700C0000087E797E790930108AB
:1015C000809300080C94661D0F931F93CF93DF93B5
:1015D0008C01FC01C081D181CE010E94131BBE0190
:1015E0000E94240DEC01B8010E942C10B801CE011C
:1015F0000E94CF0A882309F459C0B801CE010E9485
:101600007010882309F452C0B801CE010E947F0FE8
:10161000882309F44BC0C531FCE5DF0709F427C175
:10162000B0F4C130ECE5DE0709F446C008F056C05E
:10163000C115DC45B1F181E08093B2018093B30123
:10164000C801DF91CF911F910F910C94CD0AC53D38
:10165000ECE5DE0709F4F0C0B8F4C33D8CE5D8072B
:1016600009F4AEC0C43DDC4531F7F801828188231E
:1016700009F4CDC01092B3010E940C1D9093B101EA
:101680008093B00180E2A9C0C83DFCE5DF07F1F01E
:10169000C93DDC4581F6F8018281882339F082E07A
:1016A0001AC0F801828181110E94D10A80E0DF9185
:1016B000CF911F910F910895F80182818823B1F392
:1016C00080912202816080932202F0CFF801828112
:1016D000882361F380E00E94D023E8CFF801828163
:1016E000882309F4ADCF0E94321C811102C00E94F0
:1016F000181C0E944A1C90E0909341028093400283
:10170000FE01E350FC45809140028160E231F10529
:1017100038F4EC5FF64D0C94A22880914002826070
:1017200080934002809140020E944E1C0E941F162E
:10173000BDCF809140028460F3CF809140028860E9
:10174000EFCF809140028061EBCF809140028062B8
:10175000E7CF809140028064E3CF809140028068AF
:10176000DFCF809140028C60DBCF809140028E7F82
:10177000D7CF809140028D7FD3CF809140028B7F65
:10178000CFCF80914002877FCBCF809140028F7E68
:10179000C7CF809140028F7DC3CF809140028F7B65
:1017A000BFCF809140028F77BBCF80914002837F73
:1017B000B7CF90914002892F97FB87F98058B0CF1F
:1017C000F8018281882361F01092B2010E940C1D01
:1017D0009093AF018093AE0182E00E94791366CFAF
:1017E0008091B20181110FC08091AE019091AF0143
:1017F0000E94181D8639910530F486E20E944F122E
:1018000086E20E942A1382E00E9480134FCF8091CB
:10181000B30181110FC08091B0019091B1010E947C
:10182000181D8639910530F487E20E944F1287E235
:101830000E942A1380E2E8CFF801828181111ACF39
:101840008091B3018111F6CF8091B0019091B101E7
:101850000E94181D8639910568F780E20E94801366
:1018600088E20E944F1288E20E942A131FCF0E9432
:10187000D91BF8019281992381F08A7A91E009F4C9
:1018800090E09093AD01811106C089E20E94621B35
:101890000E94A61B0BCF85E3F9CF8091AD0181118A
:1018A00004C089E20E94691BF3CF85E3FBCFCF938D
:1018B00090E0FC01E053F54FC491805B944FFC0134
:1018C0008491882369F081EE0E944F128C2F0E9430
:1018D0004F128C2F0E942A1381EECF910C942A1361
:1018E0008C2F0E944F128C2FF8CFFF920F931F93D3
:1018F000CF93DF938C01F62EF8018491882349F170
:10190000E8012196813049F4FE011491812F0E9453
:101910004F12812F0E942A1306C0823089F4FE01E3
:1019200084910E944F128E010F5F1F4F8F2D8150A7
:1019300018F3EFE9FFE03197F1F700C00000F7CFAF
:10194000833019F4FE018491E5CF0E94570CE80121
:10195000EACFDF91CF911F910F91FF90089560E042
:101960000C94750C8F929F92AF92BF92CF92DF92A0
:10197000EF92FF920F931F936B017C0181E090E047
:10198000A0E0B0E04C015D0104C0880C991CAA1CC9
:10199000BB1C4A95D2F7B501A4014C015D0104C0FE
:1019A000880C991CAA1CBB1C2A95D2F748295929D6
:1019B0006A297B2904C0880F991FAA1FBB1F0A959B
:1019C000D2F78A019B010C211D212E213F210417F2
:1019D00015072607370789F48C299D29AE29BF29C9
:1019E000BC01CD011F910F91FF90EF90DF90CF9040
:1019F000BF90AF909F908F90089580959095A095FF
:101A0000B0958C219D21AE21BF21EACF0F93382FB5
:101A1000262F60910D0270910E0280910F0290911D
:101A20001002042F432F0E94B20C0F910C94511AF4
:101A30000C94A7090E94CA100C94E70608950C9410
:101A40001E0D0C941F0D0895972F70E026E0929FB5
:101A5000600D711D1124FB019CE3899FE00DF11DB8
:101A60001124EE0FFF1FE852FD4F859194910895C8
:101A7000FC01EE0FFF1FE053F44F85919491089500
:101A8000CF93DF930E94240D0E94E00EEC0181159C
:101A900020E5920708F042C0811530E4930708F072
:101AA00007C1883E910528F5803E910508F09BC04E
:101AB000883A910588F4853A910508F08AC081300A
:101AC000910509F490C0009709F48DC0049708F0BF
:101AD0008AC0D0E0C0E087C08D3B910508F487C084
:101AE000805C9109C03CD105A0F30E94380DEC0147
:101AF0007AC08115904250F4C11581E0D80708F0F2
:101B000072C0C03FD10528F3D0656DC0C11590E308
:101B1000D90708F0C3C0CE019F70E7CF811525E536
:101B2000920758F5811534E5930708F0F0C0811548
:101B300042E5940750F4C11581E5D80708F4BBC00D
:101B4000DC2FCC27C16FD06A4EC0982F9695969502
:101B50009E0123703327C115D34508F0C9C0C1E0E9
:101B6000D0E002C0CC0FDD1F2A95E2F720E2929F61
:101B7000C0011124C82BD92BB9C0C11589E5D807DC
:101B800080F4C11598E5D90708F0C6C0C11526E54F
:101B9000D20708F09ECFDC2FCC27CC27DF71D06294
:101BA00022C0CE01C1153AE5D30708F4BAC0905659
:101BB0008115904208F08DCF8D2F8F710E945B0FA1
:101BC00090E0982F882788279F719C012C2BE90192
:101BD000E6CF853A910509F4AEC0863A910509F041
:101BE000ADC0C2E8D0E4CE01DF91CF910895883A2C
:101BF000910509F4A6C0893A910509F4A5C08A3A6D
:101C0000910509F4A4C08B3A910509F4A3C08C3A5C
:101C1000910509F4A2C08B3B910509F4A1C08C3B4E
:101C2000910509F4A0C08D3A910509F49FC0803B4D
:101C3000910509F49EC08E3A910509F49DC08F3A32
:101C4000910509F49CC0813B910509F49BC0823B3E
:101C5000910509F49AC0833B910509F499C0843B2E
:101C6000910509F498C0853B910509F497C0863B1E
:101C7000910509F496C0873B910509F495C0883B0E
:101C8000910509F494C0893B910509F493C08A3BFE
:101C9000910509F492C0C0E0D4E4A5CFCE01992704
:101CA000D3FF03C0EC01D86C9ECFEC01D06C9BCF6E
:101CB000DF70D06A98CFCE01E4E096958795EA95DB
:101CC000E1F783702C2F26952695237090E2299FAB
:101CD00090011124382B8C2F8370C1E0D0E002C01A
:101CE000CC0FDD1F8A95E2F7C22BD32BDC687BCFAC
:101CF000C1E0D0E002C0CC0FDD1F2A95E2F730E250
:101D0000939FC0011124C82BD92BDA686CCFD82F30
:101D1000CC27C46FD06A67CFDC2FCC27C06FD06AC6
:101D200062CF34E0969587953A95E1F78F70CF7042
:101D3000C06ED82FBECFC1E8D0E455CFC3E8D0E401
:101D400052CFC2EED4E44FCFC9EED4E44CCFCAEEAA
:101D5000D4E449CFC5EBD4E446CFC6EBD4E443CFBB
:101D6000C3EBD4E440CFC4EBD4E43DCFC7EBD4E421
:101D70003ACFCCECD4E437CFCDECD4E434CFC3E8C5
:101D8000D5E431CFCAE8D5E42ECFC2E9D5E42BCFD4
:101D9000C4E9D5E428CFC1E2D6E425CFC3E2D6E436
:101DA00022CFC4E2D6E41FCFC5E2D6E41CCFC6E200
:101DB000D6E419CFC7E2D6E416CFCAE2D6E413CFF1
:101DC0008238910549F1B0F48133910509F462C07C
:101DD00048F48932910509F456C08A32910509F414
:101DE00060C008958533910509F446C08933910593
:101DF00099F00895833E910531F138F4803E9105C4
:101E000091F0823E9105B1F00895863E910521F151
:101E1000873E910551F10895209140022370D9F039
:101E200080EE90E008952091400220FF14C089E3E5
:101E300090E008952091400222FF0DC024FD09C0CA
:101E400083EE90E008952091400222FD31C024FFEE
:101E500002C090E080E008952091400223FFFBCF74
:101E600024FDF7CF87EE90E008952091400223FFF4
:101E7000EECF86EE90E008952091400225FFEBCF53
:101E800089E290E008952091400225FFE4CF85E3A8
:101E900090E008952091400226FFDDCF8AE290E095
:101EA00008952091400226FFD6CF81E390E0089567
:101EB00082EE90E008959091400292FF06C0282F94
:101EC0002871283069F4877F846093FF06C0282F2B
:101ED0002871283161F4877E846194FD877E08959E
:101EE000282F2471243089F78B7F8860EECF282F2C
:101EF0002471243191F78B7E8861EFCF08950F9381
:101F00001F93CF938C01FB018281811106C0C1E038
:101F10008C2FCF911F910F910895C091C101C111D4
:101F200025C006311C4599F70E947E0F81E0809301
:101F3000C1010E940C1D9093C0018093BF011092BB
:101F4000B4011092B6011092B5011092B80110922E
:101F5000B7011092BA011092B9011092BC0110920F
:101F6000BB011092BE011092BD01D2CF8091BF0182
:101F70009091C0010E94181D8C32914040F68091D2
:101F8000B401E82FF0E0EE0FFF1FEB54FE4F11837A
:101F900000838F5F8093B401C0E0BACFCF93DF930B
:101FA000EC0181E08F878F810E94DC1B88850E9475
:101FB000EF1B0E94A61BEA81FB81309739F06A89EA
:101FC0007B89CE010696DF91CF910994DF91CF9165
:101FD0000895EF92FF920F931F93CF93DF93EC013D
:101FE0008885811132C0EB80FC8087E5F81A24E1F6
:101FF0002E9DC0012F9D900D1124DC01AF5FBE4FBF
:102000001496ED91FC911597309731F052966D91A1
:102010007C91895F9E4F099584E18E9D80018F9D03
:10202000100D11240F5F1E4FF80187810E94E21BE3
:10203000F80180850E94F51B0E94A61B18821F8252
:1020400019861092C3011092C201DF91CF911F91A6
:102050000F91FF90EF900895DF92EF92FF920F9310
:102060001F93CF93DF937C01FB018281882391F042
:10207000809151018F3F71F0C1E0D1E010E000E0AC
:10208000DD24D39480915101082E000C990B801708
:10209000910744F4DF91CF911F910F91FF90EF9042
:1020A000DF9008958E818823B9F089859A858E15F1
:1020B0009F0539F48091C2019091C3018E159F054F
:1020C00059F0DD868F85811103C0CE010E94CE0FAD
:1020D000CE0106960E94E90F0F5F1F4F6496D2CF84
:1020E000EF92FF920F931F93CF93DF937C0197554D
:1020F0008F3F910509F0D8F520915101022E000C77
:10210000330B2817390714F480935101FB01228106
:1021100034E1389F8001399F100D1124E801CF5F11
:10212000DE4F2E8792818E81992349F1FA86E986C6
:102130008F5F8E830E940C1D9C878B870E94151CCD
:102140008F830E94D91B88870E94EC1B9885892B5E
:102150008887E881F981309731F06A897B89C801E5
:10216000895F9E4F0995F092C301E092C20181E020
:10217000DF91CF911F910F91FF90EF9008958823E9
:10218000B1F38F85882399F3C801895F9E4F0E9420
:10219000E90FEDCFEF92FF920F931F93CF93DF9351
:1021A0008091510110E004E18F3FC1F5DF91CF91A3
:1021B0001F910F91FF90EF900895029FF001039FF0
:1021C000F00D1124EF5FFE4FE088F188E114F10477
:1021D00019F486E9E82EF12C029FE001039FD00D4F
:1021E0001124CF5FDE4F8E818823B9F08B859C85CB
:1021F0000E94181DE816F90680F4109F7001112442
:102200008F85811105C0C7018F5F9E4F0E94CE0F41
:10221000C701895F9E4F0E94E90F1F5F212F30E0A9
:1022200080915101082E000C990B821793072CF610
:10223000BDCF9093C9018093C8010895E091C80172
:10224000F091C901309721F00190F081E02D0994BF
:1022500080E00895E091C801F091C901309721F024
:102260000280F381E02D09940895E091C801F09176
:10227000C901309721F00480F581E02D099408957B
:102280002091C6013091C7012817390771F090934A
:10229000C7018093C601E091C801F091C901309750
:1022A00021F00680F781E02D099408952091C40162
:1022B0003091C5012817390771F09093C5018093BB
:1022C000C401E091C801F091C901309721F0008468
:1022D000F185E02D099408950C94930881E0089508
:1022E0000E94031D0E94E9060C94771DBF92CF92B5
:1022F000DF92EF92FF920F931F93CF93DF93CDB7AF
:10230000DEB72A970FB6F894DEBF0FBECDBF0E948E
:1023100023080E946E11882309F471C08BECC82E2B
:1023200081E0D82E10E000E0B02E802F0E946308DC
:10233000E82EF601F1906F01F81609F45AC0809169
:10234000220281FD0E94690890E080E0FE242F2D8A
:1023500030E0482FB901082E02C0759567950A94A0
:10236000E2F760FF41C08E83BF8281E090E06C01A4
:1023700002C0CC0CDD1C4A95E2F72E2D30E02C215A
:102380003D21232B09F480E088870E940C1D816089
:10239000782F9A8789874E815F8168858A850E9418
:1023A0002012F801E553FE4F80818C2580830E9426
:1023B000051F0E941E119091CA01891789F10E9480
:1023C0001E118093CA012A960FB6F894DEBF0FBE85
:1023D000CDBFDF91CF911F910F91FF90EF90DF90D4
:1023E000CF90BF900C94210D01968630910509F095
:1023F000B0CF0F5F1F4F0A30110509F095CF8FEF57
:1024000089838A831B820E940C1D8160782F9D83A3
:102410008C8349815A816B818D810E942012C7CFA4
:102420002A960FB6F894DEBF0FBECDBFDF91CF91D5
:102430001F910F91FF90EF90DF90CF90BF90089584
:10244000CF93DF93CDB7DEB72B970FB6F894DEBFEF
:102450000FBECDBF4F83588769877A878B871E82CF
:102460001D8285E0FE013796DE01119601900D92E6
:102470008A95E1F749815A816B817C818D819E81AA
:102480002B960FB6F894DEBF0FBECDBFDF91CF9174
:102490000C94F518FC01808191810C94551BCF930D
:1024A000C82F882309F4D4C08238C1F40E941E11B9
:1024B00081FDCEC089E30E94621B0E94A61B2FEF04
:1024C00081EE94E0215080409040E1F700C0000090
:1024D00089E30E94691BCF910C94A61B8338A1F459
:1024E0000E941E1180FDB4C083E50E94621B0E9401
:1024F000A61B2FEF81EE94E0215080409040E1F741
:1025000000C0000083E5E5CF8438A1F40E941E11CD
:1025100082FD9EC087E40E94621B0E94A61B2FEFD3
:1025200081EE94E0215080409040E1F700C000002F
:1025300087E4CFCF8CEF8C0F813A48F48C2F0E9428
:102540000721811185C08C2F0E94621BC4CF80E2BD
:102550008C0F883048F4C77081E001C0880FCA959D
:10256000EAF70E94DC1BB7CF8BE58C0F833068F451
:1025700081E890E0C53A31F083E890E0C63A11F482
:1025800082E890E0CF910C94401188E58C0F853162
:1025900008F05EC082EE90E0C83A09F456C089EEB9
:1025A00090E0C93A09F451C08AEE90E0CA3A09F4C1
:1025B0004CC085EB90E0CB3A09F447C086EB90E045
:1025C000CC3A09F442C083EB90E0CB3BF1F184EBD1
:1025D00090E0CC3BD1F187EB90E0CD3AB1F18CECBF
:1025E00090E0C03B91F18DEC90E0CE3A71F183E840
:1025F00091E0CF3A51F18AE891E0C13B31F182E9B3
:1026000091E0C23B11F184E991E0C33BF1F081E23A
:1026100092E0C43BD1F083E292E0C53BB1F084E2AA
:1026200092E0C63B91F085E292E0C73B71F086E212
:1026300092E0C83B51F087E292E0C93B31F090E074
:1026400080E0CA3B11F48AE292E0CF910C945611DB
:10265000CF910895882309F44BC0823871F40E9409
:102660001E1181FF45C089E30E94621B0E94A61BC8
:1026700089E30E94691B0C94A61B833859F40E94BD
:102680001E1180FF35C083E50E94621B0E94A61BBD
:1026900083E5EFCF843859F40E941E1182FF28C0D1
:1026A00087E40E94621B0E94A61B87E4E2CF9CEF96
:1026B000980F913AF0F290E2980F983050F48770AA
:1026C00091E001C0990F8A95EAF7892F0E94E21BD9
:1026D000D2CF9BE5980F933020F490E080E00C94EB
:1026E0004011885A853120F490E080E00C94561116
:1026F0000895882321F00E94DC1B0C94A61B0895EA
:10270000882321F00E94E21B0C94A61B08958F924F
:102710009F92AF92BF92CF92DF92EF92FF920F9370
:102720001F93CF93DF937C01D62FC72FFC01058128
:1027300002950F70128111110E94FC1B0E949F1BB9
:10274000C82E882371F01123B1F080E28D0F8830FC
:1027500090F082E00E94891B0E949F1B91E0C82E8E
:10276000C926DC2ED2949FE0D922ED2DF0E0EA5E5E
:10277000F64D0C94A228C12CF4CF0C2F0F70C07F03
:1027800011F00295007F1123A9F0002359F080E297
:102790008D0F883010F0D11109C0802F0E94DC1BF2
:1027A0000E94A61B8D2F0E944F1214C0802F0E94E2
:1027B000EF1BF6CF8D2F0E942A13002359F080E2E1
:1027C0008D0F883010F0D11133C0802F0E94E21B92
:1027D0000E94A61B98E0D91639F0D91648F086E079
:1027E0008D0D8F70823020F40E941E110E94210DE9
:1027F000CC2009F4D9C10E947C1B80FDD5C1F70112
:1028000012820E94761B0E94771AC7010E94E1156E
:102810000E94761BDF91CF911F910F91FF90EF9057
:10282000DF90CF90BF90AF909F908F900C94981AAC
:10283000802F0E94F51BCCCFFC2FFF70BF2EC07FD6
:10284000C03219F0B29480EFB822DD2369F0D130A4
:1028500049F1112391F1002351F1F701858180FFA6
:10286000A1CF8F70858323C0112381F0011106C091
:102870000E94151C8B290E947913ACCF0130C1F73F
:102880000E94151C8B290E940F1CA4CF011106C0A9
:102890000E94121C8B2D0E9480139CCF013009F4E2
:1028A00099CFF6CF112329F0063008F093CF8B2D66
:1028B000E2CF053008F08ECFEDCF002359F38D2FF6
:1028C0000E942A1387CF8C2F86958695837069F096
:1028D000813009F07FCF8D2F9C2F9370111102C092
:1028E00090E080E00E94561175CF8D2F9C2F937041
:1028F000111102C090E080E00E9440116BCF1123C3
:1029000009F1D53F99F0D63FB9F0D43F49F4809111
:102910003A0290913B02816090933B0280933A028D
:102920008D2F0E94131E0E94FA1E54CF80913A02EE
:1029300090913B028260F0CF80913A0290913B02ED
:102940008460EACFD53F89F0D63FA9F0D43F49F45F
:1029500080913A0290913B028E7F90933B0280934C
:102960003A028D2F0E947B1EDECF80913A02909119
:102970003B028D7FF2CF80913A0290913B028B7F98
:10298000ECCF8C2F837009F047C0111123CF2D2F6E
:10299000229526952770220F220F6D2F6F70862E9D
:1029A000912CB12CA12C022E04C0880C991CAA1CBD
:1029B000BB1C0A94D2F760E070E0CB01D4FF0FC0DB
:1029C0006FE070E080E090E004C0660F771F881F22
:1029D000991F2A95D2F76095709580959095C69528
:1029E000C695C370C23051F080F4682979298A29CC
:1029F0009B29C13071F00E94291AECCE68297929EF
:102A00008A299B290E943B1AE5CE0E94291AC501FA
:102A1000B4010E94171ADECE8695112311F08C2F77
:102A20008170882309F4D6CE2D2F22952695277004
:102A3000220F220F6D2F6F70862E912CB12CA12C9E
:102A4000022E04C0880C991CAA1CBB1C0A94D2F745
:102A500060E070E0CB01D4FF0FC06FE070E080E079
:102A600090E004C0660F771F881F991F2A95D2F740
:102A70006095709580959095C695C695C370C23047
:102A800051F080F4682979298A299B29C13071F095
:102A90000E94EE1A9FCE682979298A299B290E94D3
:102AA000001B98CE0E94EE1AC501B4010E94DC1AE8
:102AB00091CEE0E2ED0FE53108F04DC0F0E0EA5DC7
:102AC000F64D0C94A228DF708C2F8F71112321F00A
:102AD0000E94771A8D2FCFCE0E94981A8D2FDBCEB1
:102AE000112341F0053008F075CE8C2F8F710E94B4
:102AF000BB1A70CE063008F06DCEF7CF8C2F8F71D9
:102B0000112339F00E94771A65CE8C2F8F71112313
:102B1000C9F30E94981A5ECE112329F08C2F8F7171
:102B20000E94621A57CE0E945D1A54CE112349F0BA
:102B3000CF718C2F0E94771A63E08C2F0E94801B2C
:102B400049CE81E00E94891B023008F443CE82E026
:102B50000E94891B3FCE112329F0011123CE8C2F17
:102B60008F71D0CF002369F0D93309F0A8CEFFEFE1
:102B700027EE83E0F15020408040E1F700C00000E4
:102B80009ECE8C2F8F71C5CF4C2F4F706D2FC701EC
:102B90000E94F2090E948F191DCE4C2F4F706D2F8D
:102BA000C7010E94230D16CEDF91CF911F910F9187
:102BB000FF90EF90DF90CF90BF90AF909F908F905D
:102BC00008950F931F93CF93DF93EC018B819C812A
:102BD000892B29F08881998189238F3F29F4DF91FE
:102BE000CF911F910F910895CE010E94E40A88238E
:102BF000B1F3688179818A810E945F1B8C010E94F8
:102C0000121B0E94141AB801CE01DF91CF911F91BF
:102C10000F910C9487130E94FC1B0E940C1C0E94B5
:102C2000701B0E94A61B0E948F1F0E94FA1E90E03C
:102C300080E00E94401190E080E00C9456110E94C8
:102C4000E91B0C940B160E94551BE92FE295EF70BF
:102C5000E250EE3070F4F0E0E55CF64D0C94A22802
:102C6000803F19F020F4803E20F481E00895843FF5
:102C7000E1F380E00895803EC0F3813FD1F7F5CFC6
:102C800093FB882780F90895CF93DF9300D000D07D
:102C90000F92CDB7DEB70F900F900F900F900F905F
:102CA000DF91CF910895CF93DF9300D000D000D073
:102CB000CDB7DEB726960FB6F894DEBF0FBECDBFF8
:102CC000DF91CF9108951F93CF93DF93C091D501EA
:102CD00016E08091D6018C1304C0DF91CF911F9133
:102CE0000895D0E01C9FF0011D9FF00D1124E952C2
:102CF000FE4F4081518162817381848195810E9460
:102D000053162196C770E5CF4091070250910802F3
:102D10006091090270910A0280910B0290910C025D
:102D20000C9453162091D5019091D60156E02913A9
:102D300002C080E0089530E0529FF001539FF00DF3
:102D40001124E952FE4F7181761306C07081781309
:102D500003C07281741304C02F5F3F4F2770E7CF09
:102D600081E008951F93CF93DF9380910C02807FC1
:102D7000C1F4809109028823A1F08091D501C0910E
:102D8000D601609107027091080240910A025091A9
:102D90000B02D62FD723DA01A095B09516E0C81301
:102DA00004C0DF91CF911F91089590E04115510526
:102DB00011F0DF3F31F401968770F1CF2A0F3B1FEE
:102DC00017C0189FF001199FF00D1124E952FE4F12
:102DD00021812713F0CF20812613EDCF22812111ED
:102DE000EACF238134812417350740F3241B350BA8
:102DF0002639310500F720910C022F7020612093B5
:102E00000C0226E0289FF001299FF00D1124E452C6
:102E1000FE4F80818F708061808387E092E00E9406
:102E2000E115DF91CF911F910C9463169F92AF92A1
:102E3000BF92CF92DF92EF92FF920F931F93CF93A7
:102E4000DF93CDB7DEB761970FB6F894DEBF0FBE44
:102E5000CDBF8C0185E0F801DE011D9601900D9239
:102E60008A95E1F7D801DC901196EC9011971296B3
:102E7000CC90129780910A0290910B02009709F46E
:102E800092C12091070230910802422F43234F3F05
:102E900009F489C11396AD90BC90909009029920D5
:102EA00009F422C1A816B906E0F1F501E81BF90BF7
:102EB000CF01FF24F3948639910508F0F12C80911D
:102EC0000C02982F907FFF2009F4C7C091118EC08B
:102ED000FC2C3E112BC02D1129C0C11027C08F70B2
:102EE000806180930C020E94841687E092E00E9429
:102EF000E11580910C02D80115968C938F2D619667
:102F00000FB6F894DEBF0FBECDBFDF91CF911F91FA
:102F10000F91FF90EF90DF90CF90BF90AF909F9078
:102F20000895809590958A0D9B1DC3CFA114B1047F
:102F300029F08E2D8D218F3F09F054C180E080FF54
:102F400016C04C2D6E2D8D2D0E949216882379F07F
:102F500087E092E00E94E11586E0E7E0F2E0DF0121
:102F60001D928A95E9F70E948416F12CC7CFAB28F1
:102F700029F08E2D8D218F3F09F031C180E0B82FCF
:102F8000B170AB2E80FF29C04C2D6E2D8D2D0E946F
:102F90009216B82E811121C0DD86EE868D859E8524
:102FA0000E94551B292F22952F70223050F024307B
:102FB00078F49F7051F0F8019581907F31F4FB2CEB
:102FC0009DCF9F7011F08823D1F3805E8830B8F3D5
:102FD000C8010E94E115BA2CF2CFCC2009F48ECFA3
:102FE00080910C02816080930C02BFCF3E1106C01D
:102FF0002D1104C0D801CC2009F49CC0DD86EE86DA
:103000008D859E850E942316882319F1CC2009F115
:1030100080910C02803270F02091070230910802FA
:1030200038872F831986BB86AA868C87CE010796A0
:103030000E94E11586E0F801A7E0B2E001900D9250
:103040008A95E1F70E94B2160E948416FF24F39439
:1030500055CFC8010E94E115F9CF911115C07A2D05
:10306000B98AA88A4D2D5E2D6C2D89890E9444163F
:1030700087E092E00E94E11586E0E7E0F2E0DF0100
:103080001D928A95E9F763C03E1112C02D1110C040
:10309000C1100EC0F8018583C8010E94E115E7E068
:1030A000F2E086E0DF011D928A95E9F7F92C26CF40
:1030B000DD86EE868D859E850E942316882349F243
:1030C000CC2039F280910C02803208F4B3CF2091E9
:1030D0000702309108023A8329831B82BD82AC82A9
:1030E0008E83CE010196A4CFA816B90698F1F501FA
:1030F000E81BF90BCF01F12C8639910508F049C086
:10310000FC2CCC2009F4A5CF3E1132C02D1130C0CB
:1031100080910C0280FD23C0982F907F01F1D8018F
:1031200015968C931597903F39F0982F907F905F6C
:103130008F70892B15968C93C8010E94E11586E04B
:10314000F801A7E0B2E001900D928A95E1F70E94A4
:103150008416D4CE809590958A0D9B1DCCCF86E0A9
:10316000F801A7E0B2E001900D928A95E1F7C6CE92
:10317000DD86EE868D859E850E94231681115ACFAD
:1031800080910C02816080930C02C8010E94E115BD
:10319000B5CE7A2DB98AA88A4D2D5E2D6C2D8989E0
:1031A0000E94441669CFCC2009F453CFDD86EE8609
:1031B0008D859E850E942316F82E882309F449CF19
:1031C00086E0F801A7E0B2E001900D928A95E1F760
:1031D00087E092E00E944A120E94B216B8CF81E0C6
:1031E0008C25CDCE81E08C25AACE1F93CF93DF9383
:1031F000CDB7DEB72C970FB6F894DEBF0FBECDBFAC
:103200004F83588769877A878B879C87CE0107967B
:103210000E941617882369F08A859B85892B39F0CF
:103220004F815885842F85238F3F09F071C016E0A8
:103230005FC086E0FE013796DE01119601900D9287
:103240008A95E1F78A859B85892B89F388859F81FB
:1032500089238F3F61F32091D60130E0C9010196A7
:10326000877099274091D5014817190671F40E947B
:103270001F161092D6011092D50186E0E7E0F2E029
:10328000DF011D928A95E9F7D2CF96E0929FD00197
:10329000939FB00D1124A952BE4FFE0131960190AB
:1032A0000D929A95E1F78093D6010E946316BFCFE5
:1032B000819FC001112489529E4F0E9416178823B6
:1032C000E9F0E091D5011E9FF0011124E952FE4F73
:1032D0004081518162817381848195810E9453165E
:1032E0008091D50190E00196877099278093D50150
:1032F0008091D5019091D6018913DACF2C960FB623
:10330000F894DEBF0FBECDBFDF91CF911F9108951E
:1033100069857A858B859C850E94531688CFEF92AC
:10332000FF920F931F93CF93DF938C01892B81F032
:10333000F12CEE24E394E8012196F801849184377E
:1033400070F4843008F05FC08130B1F08230A1F1B8
:10335000DF91CF911F910F91FF90EF9008958537E6
:1033600009F44CC008F43DC09CE7980F903780F7F3
:103370008F770E942A1349C00E5F1F4FFE01849170
:1033800090E2980F983060F48770FE2D01C0FF0F17
:103390008A95EAF78F2F0E94FF1B0E94A61B02C08E
:1033A0000E944F128F2D815030F2EFE9FFE03197EC
:1033B000F1F700C00000F7CF0E5F1F4FFE018491B0
:1033C00090E2980F983050F48770FE2D01C0FF0FE7
:1033D0008A95EAF78F2F0E94051CDFCF0E942A13DF
:1033E000E1CF0E5F1F4FFE01C491C150D8F28FE9AB
:1033F0009FE00197F1F700C00000F7CF0E5F1F4F6D
:10340000FE01F490CFCF0E944F128E01CBCF0895D2
:103410000E94071A609311027093120280931302A4
:10342000909314020C940B1608950C94081A0F93A1
:103430001F930091110210911202209113023091FA
:103440001402602B712B822B932B1F910F910C94E4
:10345000081A0F931F9300911102109112022091EC
:1034600013023091140260237123822393231F914E
:103470000F910C94081A0F931F9300911102109151
:1034800012022091130230911402602771278227C3
:1034900093271F910F910C94081A0C94071A0C94FF
:1034A0004D1A0E944F1A60930D0270930E02809382
:1034B0000F02909310020C940B1660E070E0CB01A9
:1034C0000C94511A0F931F9341E050E060E070E0BC
:1034D0008A019B0104C0000F111F221F331F8A9510
:1034E000D2F7C901B8011F910F910C94511A0F9393
:1034F0001F9341E050E060E070E004C0440F551FAE
:10350000661F771F8A95D2F780910D0290910E0267
:10351000A0910F02B09110028A019B01082B192B78
:103520002A2B3B2BC901B8011F910F910C94511A02
:103530000F931F9341E050E060E070E004C0440F3F
:10354000551F661F771F8A95D2F7CB01BA01609588
:1035500070958095909500910D0210910E0220912A
:103560000F023091100260237123822393231F9155
:103570000F910C94511A0F931F9341E050E060E0BB
:1035800070E004C0440F551F661F771F8A95D2F75D
:1035900080910D0290910E02A0910F02B091100245
:1035A0008A019B01082719272A273B27C901B8014F
:1035B0001F910F910C94511A0F931F9300910D02BC
:1035C00010910E0220910F0230911002602B712B8E
:1035D000822B932B1F910F910C94511A0F931F93D1
:1035E00000910D0210910E0220910F0230911002F5
:1035F00060237123822393231F910F910C94511AFE
:103600000F931F9300910D0210910E0220910F0253
:103610003091100260277127822793271F910F9105
:103620000C94511A0895BF92CF92DF92EF92FF92BD
:103630000F931F93CF93DF938C01C0900D02D09016
:103640000E02E0900F02F090100280911102909112
:103650001202A0911302B0911402C82AD92AEA2AB0
:10366000FB2ACFE1D0E0BC2ED701C6010C2E04C04E
:10367000B695A795979587950A94D2F780FD0EC0C9
:10368000219788F7B12C8B2DDF91CF911F910F914E
:10369000FF90EF90DF90CF90BF900895B8018C2FEE
:1036A0000E94400D019761F3EECFCF93DF93EC01C1
:1036B0000E94131BBE01DF91CF910C94400DCB01F2
:1036C0000C94551B682F80915201909153010C94DA
:1036D000871C682F80915201909153010C94891C92
:1036E00080915201909153010C948B1C8091150292
:1036F0008595859585950895809115028770089523
:1037000098E0899F90011124622B609315020C941C
:10371000771A909115028095892380931502282F9E
:10372000277061F4282F082E000C330B9217130614
:1037300029F08595859585950C94981A0895909112
:103740001502977081E009F480E00895E09152013C
:10375000F0915301809121028083E0915201F09118
:103760005301808190912002892B8083E091520146
:10377000F0915301808190911F02892B8083909159
:103780001602992381F0E0915201F091530180815A
:10379000892B808380915201909153010E94531C88
:1037A00081111092160280915201909153010C9454
:1037B0002A1180912102089590912102892B8093F2
:1037C00021020895809590912102982390932102DF
:1037D00008951092210208958091200208959091F9
:1037E0002002892B809320020895809590912002D9
:1037F00098239093200208951092200208959091AA
:103800001F02892B80931F020895809590911F02BB
:10381000982390931F02089510921F020895809399
:1038200016020895109216020895809116020895C6
:103830006DEE7EEF90E080E00E94DC2860E082E0A8
:1038400090E00E94CA2860E083E090E00E94CA28CD
:1038500060E084E090E00E94CA2860E085E090E0AB
:103860000C94CA2890E080E00E94C42821E08D3E9C
:103870009E4F09F020E0822F089582E090E00C94A2
:10388000BC2883E090E00C94BC28682F83E090E093
:103890000C94CA2884E090E00C94BC28682F84E043
:1038A00090E00C94CA28FC0131969C01285F3F4FA0
:1038B00080E0919191118F5FE217F307D1F708959E
:1038C0009C01FC0132969FEF80E04191461751F038
:1038D0009F3F19F4411101C0982F8F5F8630A9F7DF
:1038E0009F3F09F40895290F311D97FD3A95F9017D
:1038F00062830895FC01329608962191261303C035
:10390000DF0111971C92E817F907B9F708950C9495
:10391000601C0C947A1CFC011182128213821482A6
:10392000158216821782089580914602843039F1FB
:103930001092230288E190E020E40FB6F894A89555
:10394000809360000FBE2093600080E00E94210DF4
:1039500083B7817F846083BF83B7816083BF78949E
:10396000889583B78E7F83BF0FB6F894A895809112
:103970006000886180936000109260000FBE08951F
:1039800008950895CF930E94C01C0E9423080E94AE
:10399000C11CC0E08C2F0E946308811105C0CF5F5D
:1039A000CA30C1F7CF91089581E0FCCF0E941F1665
:1039B0000E941E110C94210D1F921FB61F921124FC
:1039C0008F939F93AF93BF9380912302811113C074
:1039D00080913C0290913D02A0913E02B0913F0245
:1039E0004196A11DB11D80933C0290933D02A0938E
:1039F0003E02B0933F02BF91AF919F918F911F9074
:103A00001FBE1F90189582E084BD93E095BD9AEF8C
:103A100097BD80936E0008952FB7F89480913C0273
:103A200090913D02A0913E02B0913F022FBF0895B8
:103A3000CF92DF92EF92FF920F931F932FB7F894DC
:103A400040913C0250913D0260913E0270913F02D4
:103A50002FBF6A017B01EE24FF248C0130E020E0BF
:103A6000C016D106E206F30650F0481B590BCA01F6
:103A70001F910F91FF90EF90DF90CF9008954150EC
:103A80005109F3CF78941F921FB61F9211248F9380
:103A90009F93AF93BF9380913C0290913D02A09180
:103AA0003E02B0913F020196A11DB11D80933C02E0
:103AB00090933D02A0933E02B0933F02BF91AF911D
:103AC0009F918F911F901FBE1F90189587E797E7D2
:103AD000909301088093000888E19AE00FB6F8946B
:103AE000A895809360000FBE90936000FFCF0E9466
:103AF000321C811102C00E94181C0E943D1C809340
:103B000022020E944A1C90E090934102809340025E
:103B10000E94411C682F70E090E080E00C94151A20
:103B20008091260280FF12C06091570185E0689F56
:103B3000B001112475956795759567956038710585
:103B4000A8F561157105A1F1862F089581FF09C0BF
:103B50006091570185E0689FB001112475956795C4
:103B6000EDCF6091570182FD0AC080912702882322
:103B7000D1F09091560160915701891728F085E0A6
:103B8000689FB0011124DACF869FB001112485E02F
:103B9000869F9001879F300D1124692F70E0C90125
:103BA0000E948E28CBCF65E070E0CECF8FE70895DE
:103BB00081E008958091260280FF0CC0609155013C
:103BC00070E075956795759567956115710549F173
:103BD000862F089581FF06C06091550170E07595AC
:103BE0006795F3CF6091550182FD0BC0909127023C
:103BF0009923A1F06091540180915501961738F0F6
:103C0000682F70E06038710500F38FE70895899F91
:103C1000C001112470E00E948E28F4CF61E070E0B2
:103C2000D7CF81E00895803F31F40E94901D8195A7
:103C300080932A020895813F19F40E94901DF8CFC5
:103C4000823F31F40E94901D81958093290208954E
:103C5000833F19F40E94901DF8CF893F29F40E94F8
:103C6000DA1D80932B0208958A3F21F40E94DA1D09
:103C70008195F7CF8B3F31F40E94DA1D81958093B7
:103C80002C0208958C3F19F40E94DA1DF8CF843F6E
:103C900031F4809128028160809328020895853F45
:103CA00021F4809128028260F7CF863F21F4809131
:103CB00028028460F1CF873F21F480912802886038
:103CC000EBCF883F21F4809128028061E5CF8D3FC2
:103CD00031F48091260281608093260208958E3F00
:103CE00021F4809126028260F7CF8F3FB9F780914F
:103CF00026028460F1CF90912902803F41F48091A7
:103D00002A0287FD10922A02992371F00895813FBB
:103D100029F480912A021816ACF3F6CF823F81F481
:103D200097FFF2CF1092290280912A0290912B02E4
:103D3000892B90912C02892B49F710922702089524
:103D4000833F19F4191674F3DFCF893F39F480915A
:103D50002B021816CCF610922B02D6CF8A3F29F4EC
:103D600080912B0287FFD0CFF6CF8B3F39F4809123
:103D70002C0287FFC9CF10922C02C6CF8C3F29F4AA
:103D800080912C021816BCF3BFCF843F31F4809190
:103D900028028E7F80932802B7CF853F21F480913F
:103DA00028028D7FF7CF863F21F4809128028B7FF8
:103DB000F1CF873F21F480912802877FEBCF883FA6
:103DC00021F4809128028F7EE5CF8D3F31F48091E0
:103DD00026028E7F8093260297CF8E3F21F480911A
:103DE00026028D7FF7CF8F3F09F08ECF809126027C
:103DF0008B7FF0CF88E292E00E9435110E940C1D6B
:103E0000909325028093240208951F93CF93DF930C
:103E100080912402909125020E94181DAC0190917E
:103E200027022091580130E0911106C020915901DC
:103E30008AE0289F900111244217530778F02091BF
:103E40002902C0912A02D0912B0210912C0221113B
:103E500009C08C2F8D2B812B09F05DC0DF91CF9194
:103E60001F9108959F3F19F09F5F909327021216AC
:103E700024F40E94901D809329028091290287FFDB
